:03000000020457A0
:030023000207B918
:03007B000205A4D7
:10007E0075D2FF75D30F75D5FF75D60F75BA00758E
:10008E00BB0075E8C5C202C203C200C201780F767A
:10009E0000781076001200261206D47811760078B9
:1000AE001576680876F712075B1207FB7819A60813
:1000BE007819E6C394557007D202D2001200267842
:1000CE0019E6C394567007C202D2001200267819A0
:1000DE00E6C394577007C202C2001200267819E6D2
:1000EE00C394757007D203D2011206D47819E6C3F1
:1000FE0094767007C203D2011206D47819E6C3941F
:10010E00777007C203C2011206D47819E6C394426F
:10011E007011780D760475D2FF75D300780F7602C4
:10012E001200267819E6C394437011780D76037584
:10013E00D2FF75D301780F76021200267819E6C326
:10014E0094447011780D760275D2FF75D303780F33
:10015E0076021200267819E6C394457011780D7652
:10016E000175D2FF75D307780F7602120026781923
:10017E00E6C394467011780D760075D2FF75D30FD5
:10018E00780F76041200267819E6C394477011781A
:10019E000D760075D2FF75D30F780F7608120026F4
:1001AE007819E6C394487011780D760075D2FF75F4
:1001BE00D30F780F76101200267819E6C394497083
:1001CE0011780D760075D2FF75D30F780F76201249
:1001DE0000267819E6C394627011780E760475D5F0
:1001EE00FF75D600781076021206D47819E6C394FD
:1001FE00637011780E760375D5FF75D6017810767B
:10020E00021206D47819E6C394647011780E760241
:10021E0075D5FF75D603781076021206D47819E6D6
:10022E00C394657011780E760175D5FF75D6077873
:10023E001076021206D47819E6C394667011780E01
:10024E00760075D5FF75D60F781076041206D47821
:10025E0019E6C394677011780E760075D5FF75D6C2
:10026E000F781076081206D47819E6C394687011C8
:10027E00780E760075D5FF75D60F781076101206AB
:10028E00D47819E6C394697011780E760075D5FF8F
:10029E0075D60F781076201206D47819E6C39430EE
:1002AE00700E78117601781576250876FF12075BA9
:1002BE007819E6C39431700E78117602781576258A
:1002CE000876FF12075B7819E6C39432700E781128
:1002DE007600781576250876FF12075B7819E6C347
:1002EE009433700E78117600781576DD0876FD124F
:1002FE00075B7819E6C39434700E78117600781582
:10030E0076B90876FB12075B7819E6C39435700E42
:10031E0078117600781576680876F712075B7819EB
:10032E00E6C39436700E781176007815769D0876B1
:10033E00EA12075B7819E6C39437700E78117600CF
:10034E007815763A0876D512075B7819E6C3943895
:10035E00700E78117600781576740876AA12075BFF
:10036E007819E6C39439700E78117600781576E810
:10037E0008765412075B7819E6C39453600302049F
:10038E0053780D86BC7811E6C3940160057811E6AA
:10039E00700A7812760008760075BB007811E6C3F5
:1003AE009402700A7812760208760075BB02D2EFBC
:1003BE00E5E74402F5E7E5914404F5917812C3E6CA
:1003CE00940008E6940830D204B2E7D2E040EDC2C1
:1003DE00EFE5E754FDF5E7E59154FBF591781276DC
:1003EE00000876007812C3E6940008E6940830D22E
:1003FE0004B2E7D2E050447812860808860918E65F
:10040E002401F608E63400F6E5082400F582E50935
:10041E003400F583781AE0F6781A791BE6F7781A25
:10042E00E6C4540F781AF6781C791AE7F6120720EC
:10043E00781C791BE7F612072080A97815760A0832
:09044E0076001207920200B722A9
:10045700758121750CFFC2D3C2D412000312051A8D
:100467001205861204FC1204DE12047C1207DA124B
:10047700007E020000740070047400601E9000008B
:10048700A883A982900000AA83AB82900000AC8366
:10049700AD82C3ED9B7028EC9A70247400700474CD
:1004A70008601B900800AC83AD82900000C3ED95F7
:1004B700827005EC95836006E4F0A30204B42288F9
:1004C700838982E493A3A883A9828A838B82F0A37A
:1004D700AA83AB820204997400600D900000790032
:1004E700FAE493F7A309DAF974086008780DFAE4D7
:1004F700F608DAFC227400600D9000007900FAE437
:1005070093F7A309DAF9740060087800FAE4F608AB
:10051700DAFC2274006035FB900000740075F00867
:10052700842420F87A08E5F06007E6031AD5F0FB83
:10053700F6EB600D1BE493A3A2E0E613F6DAF28074
:1005470005E603DAFDF6087A08EB70E57406602E17
:10055700FB740075F008842420F87A08E5F060073A
:10056700E6031AD5F0FBF6EB60091BC3E613F6DAD0
:10057700F68005E603DAFDF6087A08EB70E92274DF
:1005870000600D9000007900FAE493F7A309DAF907
:0D059700740060087800FAE4F608DAFC222F
:1005A400C0E0C082C083C0D0C008C009E8C0E0C2B7
:1005B400ED78128608088609E5082400F582E50925
:1005C4003400F583E5BFF07812740026F50808744A
:1005D4000036F509E5082401F582E5093400F583C0
:1005E400E5BEF07811E670357812E65402F5080895
:1005F400E65400F509E5084509600C75BB00780D63
:10060400E64440F5BC800A75BB02780EE64440F52A
:10061400BC7812E62402F608E63400F6187811E6EF
:10062400C39401701675BB00780DE64440F5BC78A0
:1006340012E62404F608E63400F6187811E6C394AA
:1006440002701675BB02780EE64440F5BC7812E6DB
:100654002404F608E63400F618D0E0F8D009D008EF
:09066400D0D0D083D082D0E03266
:10066D0031303338383931360050726F6475636507
:10067D0064206279207468652043726F73737761AB
:10068D007265204E6F6E2D436F6D6D65726369617E
:10069D006C2044656D6F6E73747261746F7200437C
:1006AD006F70797269676874202863292032303041
:1006BD00312043726F737377617265204173736F6D
:0706CD0063696174657300AD
:1000260078157600300011780F7915E6F73002085A
:100036007815E644017815F6C284781676007816A7
:10004600E6C3940830D204B2E7D2E0501CC283C2A1
:10005600827815E654806002D282D2837815E6C390
:0C006600337815F678160680D5D2842277
:1006D4007815760030011178107915E6F7300308A3
:1006E4007815E644017815F6C287781676007816F0
:1006F400E6C3940830D204B2E7D2E0501CC286C2EA
:10070400857815E654806002D285D2867815E6C3D2
:0C071400337815F678160680D5D28722BF
:10072000781CE6540F781DF6781DE6C3940A30D283
:1007300004B2E7D2E0500A781DE64430781DF68016
:1007400008781DE62437781DF67815791D8708E4AA
:0B075000F509A60808A609120792226E
:10075B00E5E754FEF5E775910278157917E6F7781A
:10076B00168608E4F509E50854FFF508E509540079
:10077B00F5097818A6087817869278188693781753
:07078B008694781886952280
:100792007815C3E6940A700408E6940070082005F0
:1007A200FD75990DD2052005FDD20578158699783B
:0707B20015860808860922E4
:1007B900C0E0C0D0E8C0E0309808C2987814A69983
:1007C900D204309904C299C205D0E0F8D0D0D0E063
:0107D90032ED
:1007DA0075985043A890438920438E10758BFA75FB
:1007EA008DFAD28E75910275D10375D48075D78032
:0107FA0022DC
:1000030075FFDE75FFAD75B16743B20875A4FF7563
:06001300E10443E340227A
:0D07FB003004FDC20478148608E4F50922DC
:00000001FF
